:020000040000FA
:020000000528D1
:0800080009008B13031383129E
:100010008501033083160313850004309F0003130A
:1000200083128601003083160313860003138312A4
:100030008701BF30831603138700031383128B13CA
:100040000B11030186000611061286111530E125F9
:100050003030860086158611E925F1258615861132
:100060000430E1252030BE252830BE250C30BE25C9
:100070000630BE250130BE250330E1258330BE2584
:10008000E030CE254530CE254D30CE254F30CE2523
:100090004230CE254530CE255030CE254330CE25BA
:1000A000A530CE25B130CE25C030BE257730CE2547
:1000B0007730CE257730CE252E30CE256C30CE252C
:1000C0006F30CE256330CE256B30CE252E30CE2539
:1000D0003330CE256430CE256E30CE252E30CE2561
:1000E0007230CE257530CE25640087197428B2226F
:1000F000871974286400871D7A2803138312A801C6
:10010000A901AA01AB01AC01B101BC01BD01BE0155
:10011000C7234424BC103C11BD103D11B2228610EF
:100120000610B1100317831200308C0009308D00C7
:100130002423A42203138312071DC02A871D332BF7
:10014000BA21B11C9A28A4280317831202308C000C
:1001500009308D00242303138312B1100614A42246
:1001600006107621BC1CB728BA21B11CB1289321F6
:100170003C1DBE28BA21B11CB72888280614B72315
:10018000C7232324BD11BF0106146400FF306200A1
:10019000B1109A217621BC18D42893213C19D42877
:1001A000BA21B1188828C5286400E2237621BC1C36
:1001B000DC28FD23BD14B92393213C1DE228102423
:1001C0003D15BB23FF3062000130B500A821B121ED
:1001D0009A21861406105622B11CEF28882806148E
:1001E0005622B11CF4288828B40BE628B50BE62863
:1001F0008610BD103D117621BC18022993213C19AF
:1002000002292329BF2323259A2106148614B2220A
:10021000B222B222B222B22206108610BA21B11C3A
:1002200012298828B222B222B222B222B222B222EB
:10023000B222B222B222B2227621BC180429932122
:100240003C19042923290317831201308C0009303B
:100250008D002423031383126400FF306200061410
:1002600086107621BC1C3C2993213C1D3C29382951
:100270005622B11C3C29882806107621BC1C48292E
:1002800093213C1D482944295622B11C2A2988283B
:10029000C7232324BD11BD236400FF3062009A21CF
:1002A0007621BC18D42893213C19D4285622B11C9D
:1002B0005E29B11C5E29B11C5E29882806106400E5
:1002C000FF3062007621BC18D42893213C19D42831
:1002D0005622B11C6C2988285622B11C7029882806
:1002E0005622B11C7429882806144C29BC10C2015E
:1002F00001309F0095211F1595211F197D291E088A
:10030000C100C2011E08C2009B3E03188929BC140B
:100310000800C2011E08C200963C03189129BC14B3
:100320000800BC1008003C1108000730C000C00BDA
:1003300097290800871EA2293E1D0800C323BE106E
:100340003E110800BE180800BE14C1233E15080067
:10035000BD1808007621BC1C0800FD23BD14B9237C
:1003600008003D19080093213C1D080010243D158C
:10037000BB2308009E227522962267229E228A2293
:10038000071ECF298322071EC629CF297522071EE3
:10039000CF29D121F0217623311DCF291522962294
:1003A00008003330AE000830B20096222E1CD92946
:1003B000DB298322EA290000000000000000000081
:1003C0009E228322EB2900000000000000000000B4
:1003D0000000D5299E22AE0CB20BE329832208002F
:1003E0000310203084000830B200031783128D01FF
:1003F0000313831201222D088000840AB20BFA290C
:1004000008000830B3009622000000000000000041
:100410009E228A22071E0E2AAD170F2AAD13AD0C9D
:100420008322B30B032AAD0D0800B0012D2A08303A
:10043000B00708303002031D2D2AB1109622752214
:100440008614A4228610BD190800BF0A3F08033C89
:10045000031D0800C523BD150800203084003008A6
:10046000031783128D00031383120830B2000317A1
:1004700083160C140310031783120C080313831242
:100480000002031D172A840A031783128D0A03131F
:100490008312B20B372A0030A000A100A200A300F3
:1004A000A400A500A600A700B11408006400FF3056
:1004B0006200A801A901A030AA00A80B602A642A42
:1004C000BA21B11C642A0800AA0B5D2A0800063074
:1004D000A900A800A80B6A2AA90B692A0730A9005D
:1004E000A800A80B712AA90B702A0430A900A80043
:1004F000A80B782AA90B772A0530A900A800A80B19
:100500007F2AA90B7E2A0430A900A800A80B862AFE
:10051000A90B852A00000000000000000000000078
:10052000000000006400FF3062000800071283161C
:100530000313071283120313071208008316031311
:100540000716831203130800A801A9010530AA00A9
:10055000A80BA82AA90BA82A6400FF306200AA0BE6
:10056000A82A0800A801A9010130AA00A80BB62AF0
:100570006400FF306200A90BB62AAA0BB62A080055
:100580006524B401B501071DC02AC62AB50BD02ABF
:10059000B40BD02A8614B2228610061087259A281A
:1005A000061431119E228322962267229E228A22DD
:1005B000071EC62A8322071EDE2AC62A7522071EA8
:1005C000C62AD121F0217623311DC62AE72A083018
:1005D000031783128D00031783160C14031783125D
:1005E0000C02031DF42A8C010C088D0003138312E6
:1005F0000830B200203084000317831200088C00FA
:10060000242303138312840A031783128D0A03130E
:100610008312B20BFC2A031783120D088C000313FC
:1006200083120830031783128D00242303138312CF
:1006300086140610A224B222B222B222B222B22220
:10064000B22286100614C02A831603178C130C15C9
:100650008B1355308D00AA308D008C148C182E2BE6
:100660008B170C110800C324B222B222B222B2228C
:10067000B222B222B22287196D2BB22287196D2BBA
:10068000B22287196D2BB22287196D2BB2228719DE
:100690006D2BB22287196D2B0030031783128D004A
:1006A00008308C00031383128F30B2002423031709
:1006B00083128D0A03138312B20B562B8614061471
:1006C000B22286100610A4226425B222B222B222DF
:1006D000B222B222B222B222C02AE824B222B2222C
:1006E000B222B222B222B222B2228828B60131113D
:1006F0002008B90095232108B90095232208B900E4
:1007000095232308B90095232408B90095232508CB
:10071000B90095232608B90095232708B900952329
:10072000003036020319311508000830B8003908C6
:100730003606B700370C36080318183AB700370CDE
:10074000B6000310B90C3908B80B982B08009801B3
:100750008316031398010C30990024309800C030A0
:100760008B008C1683120313803098000800000061
:100770000800000008000000080000000800000059
:100780000800000008000000080000000800013018
:10079000BE250330E1258330BE25E030CE2545302F
:1007A000CE254D30CE254F30CE254230CE2545309A
:1007B000CE255030CE254330CE25A530CE25B130C4
:1007C000CE2508000130BE250330E1258330BE254B
:1007D000E030CE254530CE254D30CE254F30CE25CC
:1007E0004230CE254530CE255030CE254330CE2563
:1007F000A530CE25B130CE2508000330E125C0302C
:10080000BE25A430CE254F30CE254830CE254130F0
:10081000CE252030CE252330CE253130CE25080000
:100820000330E125C830BE25A430CE254F30CE257B
:100830004830CE254130CE252030CE252330CE2560
:100840003230CE2508000330E125C130BE254F30BF
:10085000CE255830CE255030CE254130CE254830DB
:10086000CE254130CE252030CE254F30CE25A030AC
:10087000CE25AD30CE254530CE254B30CE2554305B
:10088000CE254130CE2508000330E125C130BE25FC
:100890004330CE254830CE25B130CE255430CE253C
:1008A0004F30CE252030CE254330CE252030CE25EA
:1008B0004F30CE255830CE255030CE254130CE2574
:1008C0004830CE25AE30CE2508000130BE2503309D
:1008D000E1258030BE252030CE25A430CE25413004
:1008E000CE25A830CE25A530CE254330CE25AD303F
:1008F000CE252030CE252030CE254B30CE25A7303A
:10090000CE25B030CE25AB30CE254530CE25A63015
:10091000CE252030CE25C330BE25E030CE25453053
:10092000CE254D30CE254F30CE254230CE25453018
:10093000CE255030CE254330CE25A530CE25B13042
:10094000CE2508000330E125C030BE252030CE255D
:100950002030CE254B30CE25A730CE25B030CE2549
:10096000AB30CE252030CE25A430CE254130CE254B
:10097000A830CE25A530CE254330CE254130CE251A
:100980004830CE2508000130BE250330E1258030F7
:10099000BE252030CE25A930CE25E030CE254130F1
:1009A000CE25A730CE25A530CE255430CE25AD306E
:1009B000CE252030CE254B30CE25A730CE25B030E9
:1009C000CE25AB30CE25A530CE253F30CE25080034
:1009D0000130BE250330E1258030BE25A930CE256B
:1009E000E030CE254130CE25A730CE254530CE256E
:1009F0004830CE25A530CE254530CE252030CE2519
:100A00002030CE254B30CE25A730CE25B030CE2598
:100A1000AB30CE254530CE25A630CE25C430BE2500
:100A20004F30CE255430CE254D30CE254530CE2505
:100A30004830CE254530CE254830CE254F30CE2506
:100A4000C030BE2508000130BE250330E1258230CC
:100A5000BE25A430CE254F30CE254830CE25AE3031
:100A6000CE252030CE252030CE254F30CE25583013
:100A7000CE255030CE254130CE254830CE25AE3063
:100A8000CE25C030BE254830CE254530CE2520307D
:100A9000CE254230CE254F30CE254330CE254330B3
:100AA000CE255430CE254130CE254830CE254F308E
:100AB000CE254230CE25A730CE254530CE25483034
:100AC000CE25AE30CE2508000330E125C030BE254E
:100AD0002030CE254B30CE25A730CE25B030CE25C8
:100AE000AB30CE25A530CE252030CE252030CE25EA
:100AF000A930CE25E030CE254130CE25A730CE25F9
:100B00004530CE254830CE25AE30CE250800013008
:100B1000BE250330E1258030BE252030CE25A4300F
:100B2000CE254130CE25A830CE25A530CE25433068
:100B3000CE25AD30CE252030CE252030CE254B30F1
:100B4000CE25A730CE25B030CE25AB30CE254530D2
:100B5000CE25A630CE25C430BE254F30CE254B3015
:100B6000CE254F30CE254830CE25AB30CE25453072
:100B7000CE254830CE254130CE2508000611BA01D9
:100B80000612BA00F0398600861586113A0EF03941
:100B90008600861586110430E12508000615BA0185
:100BA0000612BA00F03904388600861586113A0E0E
:100BB000F03904388600861586110430E1250611C7
:100BC0000800BA00F030BB00BB0BE42DBA0BE22DDD
:100BD00008001630BA000000BA0BEB2D0000000030
:0C0BE000080000000000000000000800F9
:02400E003D3F34
:00000001FF
